:100AAF007E08EE601BEFC313FFC292003091054327
:100ABF000780800353077F1EEE6002D2920080E210
:010ACF002204
:100B18007E08C292EF139291D292EFC313FFDEF2D6
:010B280022AA
:020B39008F1615
:0B0B3B00120003AF16120B18120AAFD5
:010B4600228C
:030AF100547FFD32
:100AF4008F168D17120003AF16120B18AF17020BC7
:010B040018D8
:100A89001200037FBF120B18E4FD120AAF74242D64
:100A9900F8A607EDC394085002D2920DBD09EBC226
:050AA90090C292C29111
:010AAE002225
:100AD0007515BE120003AF15120B18E4FD74242D1A
:100AE000F8E6FF120B180DBD08F3C290C292C29136
:010AF00022E3
:10099F007F8F120B39EF6007E4FD7F8E120AF47F11
:1009AF0091120B39EF6007E4FD7F90120AF47F81FB
:1009BF00120B398F15E51530E7057F80120AF17F8D
:1009CF0085120B398F15E51530E7057F84120AF173
:0109DF0022F5
:100A2000E4FD7F80120AF4E4FD7F82120AF47D0760
:100A30007F84120AF47D017F86120AF47D017F888B
:100A4000120AF47D057F8A120AF47D167F8C120A41
:0F0A5000F4E4FD7F8E120AF4E4FD7F90020AF4B5
:06000300C290C292D290EF
:020009000022D3
:100A5F00E4F597F5C1F58FF5A27591E07592E0C2B7
:100A6F0090C292C291D295F595F596F5B1F5B27502
:0A0A7F009DC075BC86C2BDC2AD2249
:100B0500E4F589F58EF58FF58A758CEEC28DD28C5C
:030B1500D2A92240
:100B2900E54B24F0F5D6E4F5D743AF04438E102204
:0D083100011300011200011400C11AC119C9
:10006600C216755D04E5B0F454036029E5B0F45496
:100076000365127041201A3E0514E514C3943240FC
:1000860035D21AE512B40104D2008027E512B40273
:1000960002D201801EC21AC219E4F520E514D394D7
:1000A600024013E512B40104D2028007E512B4023D
:1000B60002D203E4F514E5B0F45403F512E5202466
:1000C600FE604424FE606E24FC70030201A6240731
:1000D60060030203CAC200E4F55BF5133010251273
:1000E60007B3120AD0AD4A7FC2120AF4AD527FC4DA
:1000F600120AF4AD597FCC120AF4AD5C7FCE120A17
:10010600F4C21022D21022C201201026300D0D306A
:100116000E06C20EC20D8006D20E8002D20DA20DB0
:10012600E433FD7FC0120AF4A20EE433FD7FCA0257
:100136000AF4D21922C20230104CE55B14601A147C
:10014600602014602024FE602314602C24066003C3
:100156000203CAE513701B8023E5137002801D0598
:100166005B22055B22E4F513755B0522E51370023D
:10017600800AE4F513055B22E51370047513022269
:10018600E4F55BF51322055BE55BD394044004E4D8
:10019600F55B22E55B640360030203CA755B042218
:1001A600C2032010030203A9E55B14700302023C9C
:1001B6001470030202B41470030202C424FE700316
:1001C6000202E3147003020349240660030203CA11
:1001D600E5137031E52E75F00AA47C00252FFFEC9F
:1001E60035F0FEC3EF9417EE648094805011052F0E
:1001F600E52F940950030203CAE4F52F052E22E4E5
:10020600F52FF52E22E53075F00AA47C002531FF86
:10021600EC35F0FEC3EF943BEE64809480501105FC
:1002260031E531940950030203CAE4F53105302261
:10023600E4F531F53022E51364027033E53475F0E8
:100246000AA47C002535FFEC35F0FEC3EF940CEED6
:100256006480948050120535E535940950030203F5
:10026600CAE4F53575340122E4F53475350122E525
:100276003275F00AA47C002533FFEC35F0FEC3EF9F
:10028600941FEE64809480501E0533E53394095024
:10029600030203CAE4F5330532E532D3940350036F
:1002A6000203CAE4F53222E4F53275330122053839
:1002B600E538D3940750030203CA75380122053D79
:1002C600E53DD3940950030203CAE4F53D053CE538
:1002D6003CD3940950030203CAE4F53C22E51370AB
:1002E60031E54275F00AA47C002543FFEC35F0FEAB
:1002F600C3EF9417EE6480948050110543E5439450
:100306000950030203CAE4F543054222E4F543F526
:100316004222E54475F00AA47C002545FFEC35F041
:10032600FEC3EF9417EE6480948050110545E545B1
:10033600940950030203CAE4F545054422E4F54551
:10034600F54422E513702EE54675F00AA47C0025D7
:1003560047FFEC35F0FEC3EF9417EE6480948050AF
:100366000E0547E5479409405BE4F547054622E458
:10037600F547F54622E54875F00AA47C002549FFB5
:10038600EC35F0FEC3EF943BEE64809480500E058E
:1003960049E5499409402DE4F549054822E4F54923
:1003A600F54822300906E4F54DF54E22B211A211A8
:1003B600E433FD7FC6120AF4D208301104E4F5577F
:0503C600227557012221
:10083E001462C0F9A4B0999282F880908883C6A100
:06084E00868EFFBF8B9CAB
:10054000EF7029ED64016003BD0207A20AB39214A3
:10055000803ABD0313201010300D0D300E06A20A94
:1005600092148028C2148024D2148020EF64016089
:1005700003BF0507BD0104C2148011BF060CED6462
:10058000016003BD0204C2148002D214EFC39402BE
:100590005008ED7005EB70027B10301035300A32D8
:1005A00020192FE5132DFEEFC394024006EFD394DC
:1005B000044010EEC394024006EED3940340047B43
:1005C00010800FBF0207BD02047B108005BF03022D
:1005D0007B1074622BF8E6201406547FF5618002CC
:1005E000F561BD021CE5615438131313541FFFE578
:1005F0006154C04FFFE561540733333354F84FF56E
:0306000061AF6186
:0106030022D4
:10085400015564024F0190015A1A015D04015114BB
:10086400015EC81C2E101010101010101010101063
:1008740010020001061000130C00080202101010F0
:1008840010C10AC194C195C10CC110C117C108C1DE
:0B08940009C10EC118C116C191C1932B
:1003CB00120A5F120B05C2AF12099FE5B0F454037A
:1003DB0024FE601F14601F2402701E7FC9120B398C
:1003EB00EF24FF9213B213A213E433FD7FC8120A5A
:1003FB00F48006008003120A20E5B0F45403600871
:10040B0075A04043B03C80F1120732D2AF300B3AAB
:10041B00C20BE560AE5F7806C333CE33CED8F9FF9F
:10042B007C027D7D120905C3744C9FF554E49EF547
:10043B0053FEAF547C007D0A1209058F3EAE53AFBD
:10044B00547C007D0A1209058D3F3015472010445E
:10045B00C215C2AF120A89D2AF1208A0755EC87559
:10046B00BC8FD2AD300EE32009E0E559B526DBE5B4
:10047B005CB525D6E524C3940550CFD209754D0044
:10048B00754E3BA2119212C211A20D920FC20DE436
:10049B00F55B80B6300C0312002E3016031200668B
:1004AB00200D03020418852656E54AC395525018B1
:1004BB00E54A14FFE556C39F400AE5569552500492
:1004CB00D218804FC218804BE54AD395524017E59E
:1004DB00569552400DE54A14FFE5569F5004C2183D
:1004EB008031D218802DE54A65527027300E04C238
:1004FB00188020E5527009E556B42304D2188013F6
:10050B00E552D39400400AE55214B55604D2188034
:10051B0002C218301807E525B45902D21720170369
:10052B00020418E5256003020418C217F55BD20814
:05053B00F55702041851
:10002E00301121E55A6004155A8019055BE55BD342
:10003E0094044008E4F55B755A1A8008E55BB40336
:0D004E0003755B04C20C754F0175509022C4
:03000B00020604E6
:10060400C0E0C0F0C083C082C0D075D00843B03C05
:10061400E55B25E025E0242E252DF8E6FBAD2DAF86
:100624005B1205408FA0E52D2402FF7401A80F087A
:100634008002C333D8FCF452B0052DE52DD39403C6
:100644004003752D00301303120B2920100EE550C2
:10065400454F6008E55015507002154FE550454F61
:100664007002D20CD5580575BC8ED2ADD5550BB2DF
:100674000A755564301903752008200803300903EE
:1006840012095AE55E6004155E8002D215E55D60CC
:1006940004155D8002D216D0D0D082D083D0F0D0A1
:0206A400E03242
:03001B0002001EC2
:08001E00C28E43B03CC2AB32BC
:03002B000209E0E7
:1009E000C0E0C0F0C0D075D00853BCEFC2ADE5BCCC
:1009F000540724F9600C047020E5BDC4540FF54B76
:100A00008017AFBDEF75F004A4FFADBEEF4DFFE55D
:100A1000F05403F55F8F60D20BD0D0D0F0D0E0322D
:0300630002000E8A
:0A000E00538EEF43B03C53AFFB32BA
:100732007FC1120B39EF24FF920D7FC3120B398F49
:100742004A7FC5120B398F52E54A5430C4540FF513
:1007520042E54A540FF543E5525430C4540FF54470
:10076200E552540FF5457FC7120B39EF24FF921162
:100772007FC9120B39EF24FF92137FCB120B39EF93
:1007820024FF920E7FCD120B398F597FCF120B3976
:100792008F5CE5595430C4540FF546E559540FF5B2
:1007A20047E55C5470C4540FF548E55C540FF549B5
:0107B2002224
:1008A000E4F51553263FE5265430C4540FF52EE5E4
:1008B00026540FF52FE5255470C4540FF530E52567
:1008C000540FF531E5275430C4540FF532E5275461
:1008D0000FF533E5285410C4540FF534E528540FB0
:1008E000F535753610753711E5295407F538753922
:1008F00011753A02E4F53BE52AC4540FF53CE52AAC
:04090000540FF53D5E
:0109040022D0
:1007B300E52EB41003E4F52EE532B41003E4F5326C
:1007C300E4F524E530C454F02531547FF525E52EB6
:1007D300C454F0252F543FF526E532C454F0253395
:1007E300543FF527E534C454F02535541FF528E567
:1007F300385407F529E53CC454F0253DF52AE4F5C2
:100803002BE542C454F02543543FF54AE544C45410
:10081300F02545543FF552E546C454F02547543F6F
:0E082300F559E548C454F02549547FF55C2290
:10095A00E54C6003154C22C295E5516003155122FE
:10096A00D29575511430080DE55760061557754C28
:10097A001922C2082230091CE54E454D600CE54E8D
:10098A00154E7002154D754CC822C209A20F920D60
:05099A00A212921122DF
:030000000206A64F
:0C06A600787FE4F6D8FD7581750206ED42
:10090500BC000BBE0029EF8DF084FFADF022E4CCD6
:10091500F875F008EF2FFFEE33FEEC33FCEE9DEC9F
:10092500984005FCEE9DFE0FD5F0E9E4CEFD22EDE5
:10093500F8F5F0EE8420D21CFEADF075F008EF2F2F
:10094500FFED33FD4007985006D5F0F222C398FD20
:050955000FD5F0EA22BD
:1006B2000203CBE493A3F8E493A34003F68001F290
:1006C20008DFF48029E493A3F85407240CC8C33349
:1006D200C4540F4420C8834004F456800146F6DF18
:1006E200E4800B0102040810204080900831E47E6F
:1006F200019360BCA3FF543F30E509541FFEE4930D
:10070200A360010ECF54C025E060A840B8E493A3D3
:10071200FAE493A3F8E493A3C8C582C8CAC583CAFE
:10072200F0A3C8C582C8CAC583CADFE9DEE780BEB6
:01089F000058
:00000001FF
